:100000000C9462000C948A000C948A000C948A0070
:100010000C948A000C948A000C948A000C948A0038
:100020000C948A000C948A000C948A000C948A0028
:100030000C948A000C948A000C948A000C948A0018
:100040000C94E0010C948A000C948A000C948A00B1
:100050000C948A000C948A000C948A000C948A00F8
:100060000C948A000C948A000000000024002700F1
:100070002A0000000000250028002B0000000000DE
:1000800023002600290004040404040404040202DA
:100090000202020203030303030301020408102007
:1000A0004080010204081020010204081020000012
:1000B0000008000201000003040700000000000027
:1000C0000000230511241FBECFEFD8E0DEBFCDBF57
:1000D00011E0A0E0B1E0E6EFFAE002C005900D9279
:1000E000A631B107D9F721E0A6E1B1E001C01D9228
:1000F000A537B207E1F710E0C2E6D0E004C02197CF
:10010000FE010E947305C136D107C9F70E942A0279
:100110000C9479050C940000833081F028F4813030
:1001200099F08230A9F008958730A9F08830C9F09D
:100130008430B1F4809180008F7D03C08091800075
:100140008F7780938000089584B58F7784BD08955C
:1001500084B58F7DFBCF8091B0008F778093B00006
:1001600008958091B0008F7DF9CFCF93DF93282F32
:1001700030E0F901E255FF4F8491F901E656FF4F57
:10018000D491F901EA57FF4FC491CC23A1F081111A
:100190000E948C00EC2FF0E0EE0FFF1FE458FF4FA1
:1001A000A591B491EC91ED2381E090E009F480E019
:1001B000DF91CF91089580E090E0FACF1F93CF9325
:1001C000DF93282F30E0F901E255FF4F8491F901C8
:1001D000E656FF4FD491F901EA57FF4FC491CC2363
:1001E000A9F0162F81110E948C00EC2FF0E0EE0F89
:1001F000FF1FEE58FF4FA591B4918FB7F894EC9183
:10020000111108C0D095DE23DC938FBFDF91CF9111
:100210001F910895DE2BF8CFCF93DF9390E0FC0180
:10022000E656FF4F24918A579F4FFC018491882303
:10023000D1F090E0880F991FFC01E859FF4FA5917C
:10024000B491FC01EE58FF4FC591D491623071F426
:100250009FB7F8943C91822F809583238C93E881FB
:100260002E2B28839FBFDF91CF9108958FB7F894ED
:10027000EC912E2B2C938FBFF6CF8E508064809301
:100280007C0080917A00806480937A0080917A006B
:1002900086FDFCCF809178009091790008952F928F
:1002A0003F924F925F926F927F928F929F92AF9206
:1002B000BF92CF92DF92EF92FF920F931F93CF9353
:1002C000DF934B015C01842F3901E7019881911183
:1002D0003FC0F80140815181628173811401250181
:1002E000241A350A460A570AB201A10177FD1DC03A
:1002F00061E00E94DE0081E08883F60180829182C5
:10030000A282B382F80180819181A281B381F3013D
:100310004081518162817381840F951FA61FB71F91
:10032000F80180839183A283B383DF91CF911F91E2
:100330000F91FF90EF90DF90CF90BF90AF909F9084
:100340008F907F906F905F904F903F902F90089587
:10035000F6014081518162817381841A950AA60A4F
:10036000B70AF5E08F169104A104B104F0F260E041
:100370000E94DE001882D9CF8A3A910594F0843524
:1003800021E092078CF08E3F21E0920784F0883ABA
:1003900022E092077CF0823593407CF080E190E08F
:1003A000089581E090E0089582E090E0089583E070
:1003B00090E0089584E090E0089588E090E008954A
:1003C0001F920F920FB60F9211242F933F938F938A
:1003D0009F93AF93BF938091710190917201A0910F
:1003E0007301B09174013091700123E0230F2D3718
:1003F00058F50196A11DB11D2093700180937101E4
:1004000090937201A0937301B093740180916C0179
:1004100090916D01A0916E01B0916F010196A11DA7
:10042000B11D80936C0190936D01A0936E01B09308
:100430006F01BF91AF919F918F913F912F910F903D
:100440000FBE0F901F90189526E8230F0296A11D4E
:10045000B11DD2CF789484B5826084BD84B58160AB
:1004600084BD85B5826085BD85B5816085BD80917F
:100470006E00816080936E001092810080918100F7
:1004800082608093810080918100816080938100EF
:10049000809180008160809380008091B1008460B1
:1004A0008093B1008091B00081608093B000809112
:1004B0007A00846080937A0080917A0082608093D1
:1004C0007A0080917A00816080937A0080917A002E
:1004D000806880937A001092C10062E084E00E94FC
:1004E0000C0161E083E00E940C0161E089E00E9460
:1004F0000C0161E08AE00E940C0161E08BE00E9447
:100500000C0161E081E10E940C0160E083E00E9447
:10051000DE0060E089E00E94DE0060E08AE00E9488
:10052000DE0060E08BE00E94DE0060E081E10E947E
:10053000DE00E0E02E2EE0E03E2E8FB7F8948090B3
:10054000710190907201A0907301B09074018FBFFF
:1005500084E00E94B50010926A0110926B019091A4
:100560006901891751F0809369018092640190922A
:100570006501A0926601B09267018091640190913B
:100580006501A0916601B0916701B501A401481B06
:10059000590B6A0B7B0B8091600190916101A091D6
:1005A0006201B091630184179507A607B707B0F4FD
:1005B0009091680180916901981781F0809368019A
:1005C000911103C021E0813009F020E020936A01FD
:1005D000913009F4811190E090936B0180916B014F
:1005E000882309F495C040911A0150911B01609134
:1005F0001C0170911D0140931601509317016093E7
:1006000018017093190180911E0190911F01A09112
:100610002001B091210180931A0190931B01A093B6
:100620001C01B0931D018091220190912301A091A2
:100630002401B091250180931E0190931F01A09386
:100640002001B09321018092220190922301A09277
:100650002401B092250180912601843018F48F5F27
:100660008093260180912601843008F451C09501C1
:100670008401041B150B260B370BC901B80123E0BD
:1006800030E040E050E00E94420569017A011BE041
:10069000C116D104E104F10428F474E1C72ED12C71
:1006A000E12CF12CC0920C01D0920D01E0920E01D0
:1006B000F0920F018092580190925901A0925A0134
:1006C000B0925B01A0911201B0911301A7019601B4
:1006D0000E943705680D791D8A1D9B1D60933F019F
:1006E000709340018093410190934201A0911001C9
:1006F000B09111010E943705680D791D8A1D9B1D5F
:1007000060933B0170933C0180933D0190933E01C7
:100710008EE00E943D010E94BC013C0190931501B6
:10072000809314018FE00E943D010E94BC012C01C6
:10073000909313018093120180E10E943D010E9479
:10074000BC01EC019093110180931001C0900C0149
:10075000D0900D01E0900E01F0900F01930150E058
:1007600040E0C701B6010E9442052115310541054F
:10077000510509F431C120930801309309014093D8
:100780000A0150930B01D201A70196010E9437057F
:100790006093040170930501809306019093070113
:1007A000DE010E9437056093000170930101809380
:1007B0000201909303012601370162E07694679469
:1007C000579447946A95D1F740925C0150925D012D
:1007D00060925E0170925F01809158019091590181
:1007E000A0915A01B0915B0195018401081B190B7E
:1007F0002A0B3B0BD901C8018C159D05AE05BF0521
:1008000008F46AC08092580190925901A0925A014E
:10081000B0925B0161E083E00E94DE00109257011C
:100820008092530190925401A0925501B0925601CA
:1008300080924F0190925001A0925101B0925201CA
:100840008091470181110BC0C0924301D0924401B5
:10085000E0924501F092460111E01093470180912A
:10086000430190914401A0914501B0914601C81601
:10087000D906EA06FB0681F18091040190910501F9
:10088000A0910601B0910701880D991DAA1DBB1DFD
:1008900080933F0190934001A0934101B0934201A6
:1008A0008091000190910101A0910201B09103019A
:1008B000880D991DAA1DBB1D80933B0190933C019F
:1008C000A0933D01B0933E01C0924301D0924401F8
:1008D000E0924501F092460183E00E94B500019745
:1008E000C1F48091580190915901A0915A01B091A1
:1008F0005B01A5019401281B390B4A0B5B0BDA0144
:10090000C9010A97A105B10520F060E083E00E94CB
:10091000DE0086E3C82E81E0D82E9AE3E92E91E02E
:10092000F92E0FE411E028E031E049E0C501B401FF
:100930000E944F0121E3C22E21E0D22E35E3E32EA7
:1009400031E0F32E0FE311E024E031E04AE0C5018D
:10095000B4010E944F014CE2C42E41E0D42E50E37A
:10096000E52E51E0F52E0BE311E020E031E04BE005
:10097000C501B4010E944F01C0915701C43028F550
:1009800080912B0181112DC08091530190915401D0
:10099000A0915501B091560195018401081B190BD6
:1009A0002A0B3B0BD901C801B7FD0FC061E081E103
:1009B0000E94DE0011E010932B018092270190929B
:1009C0002801A0922901B0922A012114310409F4CE
:1009D000B4CD0E940000B1CD21E030E040E050E015
:1009E000CACE8091270190912801A0912901B09150
:1009F0002A01881A990AAA0ABB0A25E082169104DC
:100A0000A104B10410F360E081E10E94DE001092C5
:100A10002B01CF5FC0935701C430B9F280915301CD
:100A200090915401A0915501B0915601840D951DEE
:100A3000A61DB71D8093530190935401A0935501B7
:100A4000B0935601C2CFE0E6F1E082E390E0A0E08F
:100A5000B0E080839183A283B383148215821682CF
:100A6000178281E0808781871286138608950E940D
:100A70006405A59F900DB49F900DA49F800D911DBE
:100A800011240895A1E21A2EAA1BBB1BFD010DC063
:100A9000AA1FBB1FEE1FFF1FA217B307E407F5072E
:100AA00020F0A21BB30BE40BF50B661F771F881F0A
:100AB000991F1A9469F760957095809590959B01A0
:100AC000AC01BD01CF010895A29FB001B39FC00149
:100AD000A39F700D811D1124911DB29F700D811D6A
:100AE0001124911D0895EE0FFF1F0590F491E02D44
:060AF0000994F894FFCF09
:100AF600F4010000F4010000F4010000F40100001C
:060B0600010001000100E6
:00000001FF
